:100000000C9434000C9449000C9449000C94490061
:100010000C9449000C9449000C9449000C9449003C
:100020000C9449000C9449000C9449000C9449002C
:100030000C9449000C9449000C9449000C9449001C
:100040000C9449000C9449000C9449000C9449000C
:100050000C9449000C9449000C9449000C944900FC
:100060000C9449000C94490011241FBECFEFD4E03A
:10007000DEBFCDBF11E0A0E0B1E0E2E8F1E002C0F8
:1000800005900D92A032B107D9F70E9471000C942F
:10009000BF000C9400001092C50083E38093C4005D
:1000A000E0ECF0E080818D7F808386E08093C20069
:1000B00088E08093C10008959091C00095FFFCCF27
:1000C0008093C60080E090E00895CF93DF93EC0129
:1000D0008991882319F00E945C00FACFDF91CF91BB
:1000E000089581E087B90E944B002FEF3DE389E43A
:1000F000215030408040E1F700C0000080E091E0F6
:100100000E94650083E091E00E94650080E00E940B
:100110005C0087E091E00E9465008BE191E00E9425
:10012000650087E091E00E9465008BE191E00E940C
:10013000650087E091E00E9465008BE191E00E94FC
:10014000650087E091E00E9465008BE191E00E94EC
:10015000650087E091E00E9465008BE191E00E94DC
:10016000650091E088B1892788B92FEF34E38CE0EE
:10017000215030408040E1F700C00000F3CFF894F8
:02018000FFCFAF
:10018200434C004453530054542A204C6F7665204C
:100192002053696C766961202A0A00545254000087
:00000001FF
